:020000040800F2
:10000000E808002029020008FF140008471400082F
:10001000FD1400081F0400088116000800000000FD
:1000200000000000000000000000000003150008B0
:100030002104000800000000011500080515000853
:10004000430200084302000843020008430200087C
:10005000430200084302000843020008430200086C
:10006000430200084302000843020008430200085C
:10007000430200084302000843020008430200084C
:10008000430200084302000843020008430200083C
:10009000430200084302000843020008430200082C
:1000A000430200084302000843020008430200081C
:1000B0004302000843020008AD150008430200088F
:1000C00043020008430200084302000843020008FC
:1000D00043020008430200084302000843020008EC
:1000E00043020008430200084302000843020008DC
:1000F00043020008430200084302000843020008CC
:1001000043020008430200084302000843020008BB
:1001100043020008430200084302000843020008AB
:10012000430200084302000843020008430200089B
:10013000430200084302000843020008430200088B
:10014000430200084302000843020008430200087B
:10015000430200084302000843020008430200086B
:10016000430200084302000843020008430200085B
:100170004302000843020008430200080000000098
:10018000430200084302000800F002F800F03CF8C7
:100190000AA090E8000C82448344AAF10107DA45E2
:1001A00001D100F031F8AFF2090EBAE80F0013F0F8
:1001B000010F18BFFB1A43F0010318471C1500007C
:1001C0003C150000103A24BF78C878C1FAD852070D
:1001D00024BF30C830C144BF04680C6070470000C1
:1001E0000023002400250026103A28BF78C1FBD840
:1001F000520728BF30C148BF0B6070471FB501F0E0
:1002000059FA1FBD10B510BD00F0CFF81146FFF729
:10021000F5FF01F046FA00F0EDF803B4FFF7F2FF46
:1002200003BC00F0F5F80000094880470948004782
:10023000FEE7FEE7FEE7FEE7FEE7FEE7FEE7FEE796
:10024000FEE7FEE704480549054A064B70470000F3
:100250009D15000889010008E8020020E808002038
:10026000E8040020E804002053EA020C00F0698052
:100270002DE9F04B4FF00006002B1FBFB3FA83F5BA
:1002800003FA05F424FA05F65E4012BF1643B2FAEB
:1002900082F502FA05F4C5F120051EBF22FA05FC1D
:1002A00044EA0C04203556EA044C4FEA144418BFC3
:1002B000641C4FF000084FF00009904271EB030CF2
:1002C00039D3002919BFB1FA81F701FA07F6B0FA5C
:1002D00080F700FA07F6C7F120071EBF20FA07FCD7
:1002E00046EA0C062037B6FBF4FCA7EB0507103FE7
:1002F00007F01F0BCBF120060CFA0BFB2CFA06F6CD
:1003000044BFB3460026202FA4BF5E464FF0000B2B
:100310005BEA060C08BF4FF0010B19EB0B09ABFBB6
:10032000027C48EB0608C01B06FB02CC0BFB03CC8F
:1003300071EB0C01C1E70B46024641464846BDE859
:10034000F08B13B54FF000004FF00001AFF30080C9
:10035000BDE81C4070474FF0000200B513469446BC
:100360009646203922BFA0E80C50A0E80C50B1F10D
:100370002001BFF4F7AF090728BFA0E80C5048BF21
:100380000CC05DF804EB890028BF40F8042B08BFBF
:10039000704748BF20F8022B11F0804F18BF00F8BB
:1003A000012B7047704770477047754600F02CF876
:1003B000AE4605006946534620F00700854618B052
:1003C00020B5FFF73FFFBDE820404FF000064FF09B
:1003D00000074FF000084FF0000B21F00701AC467A
:1003E000ACE8C009ACE8C009ACE8C009ACE8C00999
:1003F0008D46704710B50446AFF300802046BDE837
:100400001040FFF70ABF0000004870478802002034
:1004100001491820ABBEFEE7260002007047FEE748
:1004200070470000F0B500231A464FF0004544F233
:10043000F45600BF016903EB830401EBC4010A60B9
:100440004A608A60CA600A620D604A624E604F6804
:1004500027F000474F6000EB8307032BB96406D2F7
:100460004FF0280C07690CEBC4043C4400E004691D
:10047000CC605B1C042BDDD3C26502668266C2665B
:1004800082650169006800F58050C160F0BD70B5FB
:10049000A4B00024012506468DF828408DF80450AC
:1004A0001494A8038DF8564005908DF810500294CE
:1004B0008DF85440C0108DF811508DF81F408DF804
:1004C000204006908DF81E508DF80F4009948DF84D
:1004D0001C4012948DF84C408DF8554069463046CA
:1004E00000F082F88DF881508DF880408DF88240C0
:1004F00028041B908DF8685080011F908DF8705073
:100500008DF8885040128DF871501E941D908DF812
:100510007250239421948DF8895019A9304619946A
:1005200000F002F824B070BD70B50C4601680546B5
:1005300001F5805188692B4A1040227BEAB30022E2
:10054000637B920642EA4362637FBBB35FF00003C2
:1005500042EA0352A37B42EA435263691A43237F70
:1005600042EAC312A37F42EA8312236A1A4394F831
:10057000243042EA830202438A61286800F58050F1
:100580008669012000F0AEF8286800F58050866189
:10059000A169A06822790843216941EA42610843C0
:1005A00094F8251040EAC110A16A40EA8100216850
:1005B000084340F40001286801E00FE010E000F576
:1005C00080500160286800F580500468012000F028
:1005D00089F8286800F58050046070BD0122AFE7FB
:1005E0000123B5E7233FDEF870B5026805460C46E7
:1005F00010683A49237C0840A168002B63D000238F
:1006000041EAC351637C002B5FD00023E67F9B054A
:1006100043EA0643194363691943A37FF3B30023F5
:1006200041EA4331237F41EA0331A3691943237926
:1006300041EA832194F820308BB3002341EA43211F
:10064000E37B41EAC311636A194394F8283041EA15
:1006500003110143116028680668012000F042F888
:10066000286806602A6890694FF641710840A36CBB
:10067000216D41EA034194F84C3063B3002394F8B0
:100680005560DB01012E00D0002643EAC603194362
:1006900094F85630012B00D0002301E017E018E059
:1006A00041EA830194F85430012B00D0002341EA41
:1006B00043010143916128688469012000F012F828
:1006C0002868846170BD01239AE701239EE7012316
:1006D000A6E70123B2E70123D1E700000F8120FF45
:1006E00072B6FEE770B5044600F0FEF90546601CE0
:1006F00002D004480078044400F0F6F9401BA04200
:10070000FAD370BD08000020F8B5040003D0D4F877
:10071000840010B107E00120F8BD2320C4F8840054
:10072000204600F07DF83B480025016841F48041F7
:100730000160006800F4804000903748016821F4AF
:10074000000101600168A26811430160006820682F
:1007500000F58050016841F00101016000F0C4F92A
:1007600006464FF4FA770BE000F0BEF9801BB84262
:1007700006D90420C4F88800E020C4F88400CAE741
:10078000206800F580500068C007EDD12046FFF7D3
:100790007EFE0021E06801EB810200EBC2000560F3
:1007A00045608560C56004EB81039861036843F48C
:1007B00080130360032905D22826E36806EBC202F2
:1007C0001A4400E0E268C260026842F4400202603B
:1007D000491C0429DED3A5622068E16800F5805039
:1007E00001612046FFF71EFE60680C4A8188116493
:1007F0000178C37841EA0361837840781B0443EAB7
:10080000002001435164C4F888501020C4F88400CB
:100810000020F8BD44380240043801400080024006
:10082000F0B587B0044614216846FFF794FD2D49C2
:100830002068884253D12C480024016841F000719F
:100840000160016801F000710591016841F080616B
:100850000160016801F080610591016841F000616B
:100860000160016801F000610591016841F0040137
:100870000160016801F004010591016841F0010186
:100880000160016801F001010591016841F0020178
:1008900001600068022500F0020005903220CDE9D9
:1008A000000502AA03260B2782E8D00069460F48FC
:1008B00000F022F88620CDE9000502AA694682E808
:1008C000D0000B4800F018F84FF46050CDE9000557
:1008D00002AA694682E8D000064800F00DF807B089
:1008E000F0BD0000008002403038024000080240A5
:1008F00000000240000402402DE9F84FDFF8BCA1DF
:100900000022012503264FF00F090AF1040BAAF17A
:10091000040E00BF0B6805FA02F42340A34270D115
:100920000F7907F00307012F01D0022F16D1876836
:100930004FEA420806FA08FC27EA0C07D1F80CC077
:100940000CFA08FC4CEA070CC0F808C04768A7433B
:100950000C79C4F3001494403C4344600C79E443A4
:10096000A4070AD0C4684FEA420C06FA0CF7BC434D
:100970008F6807FA0CF72743C7600C7904F003046B
:10098000022C12D1D40800EB840CDCF8204057076D
:10099000FF0E09FA07F824EA0804D1F8108008FAD3
:1009A00007F848EA0408CCF8208004684FEA420CB3
:1009B00006FA0CF7BC430F7907F0030707FA0CF7A8
:1009C000274307604C6814F4403F70D03C4C2768C4
:1009D00047F480472760246822F0030704F480442A
:1009E0000094384C07EB040CDCF8084897074FEAF2
:1009F000177809FA08F7BC43334FB84202D10027F1
:100A000024E054E0314FB84201D101271EE0304FBD
:100A1000B84201D1022719E02E4FB84201D1032775
:100A200014E02D4FB84201D104270FE02B4FB842FC
:100A300001D105270AE02A4FB84201D1062705E077
:100A4000284FB84201D1072700E0082707FA08F726
:100A50002743CCF80878DAF800405746D1F804C0AC
:100A60009C435FEACC2C00D51C433C60DBF8004083
:100A70005F46D1F804C09C435FEA8C2C00D51C4330
:100A80003C60DEF800407746D1F804C09C435FEA42
:100A90008C3C00D51C433C60084F083F3C68D1F8B3
:100AA00004C09C435FEACC3C00D51C433C60521C14
:100AB000102AFFF42FAFBDE8F88F0000083C01407A
:100AC000443802400030014000000240000402406F
:100AD00000080240000C02400010024000140240D6
:100AE00000180240001C0240014880687047000066
:100AF0000800002002488168027811448160704734
:100B0000080000200B4810B5016841F40071016035
:100B1000016841F480610160016841F48071016005
:100B2000032000F09BF80F2000F006F800F050F8CA
:100B3000002010BD003C024030B505461F4887B07C
:100B40000024016841F004010160006806A900F07A
:100B50000400009001A800F02DF90498A8B100F05D
:100B600049F940001649174AB0FBF1F11648491EF1
:100B7000026040F2E732C0E90324C0E90114846155
:100B800000F032FB040003D015E000F033F9E9E790
:100B90000D4800F057FB04000DD11E2000F030F886
:100BA000102D07D2002229461E2000F037F80748F2
:100BB000056000E0012407B0204630BD4038024007
:100BC00040420F0000080040400200200C000020BE
:100BD0000A4808B5016841F480410160006800F4EA
:100BE000804000900548001F016841F0805101607D
:100BF000006800F08050009008BD000044380240BA
:100C0000002809DB00F01F0201219140400980000B
:100C100000F1E020C0F8001170470000F0B40E4B66
:100C20001B680C46C3F30223C3F10705042D00D94A
:100C30000425191D072901D2002300E0DB1E01262F
:100C400006FA05F1491E214099409E40761E164045
:100C50003143F0BC00F015BD0CED00E0064900F09A
:100C6000070208684FF6FF03184040EA0220034AD3
:100C700010430860704700000CED00E00000FA052A
:100C80002DE9F0470E46050065D0DFF81481D8F84D
:100C90000000F7B200F00700B04207D288F80070F9
:100CA000D8F8000000F00700B04254D128683D4C4D
:100CB000810712D5400703D5206840F4E05020603A
:100CC0002878000703D5206840F460402060206841
:100CD000A96820F0F000084320602878C0072DD0D4
:100CE000304968680839012812D0022813D0032837
:100CF00011D00968890700292DDA216821F0030144
:100D000001432160FFF7F0FE814641F2883A0EE090
:100D100009688903EFE709688901ECE7FFF7E4FE5A
:100D2000A0EB0901514502D90320BDE8F0872068F6
:100D3000696800F00C00B0EB810FEFD1D8F800101B
:100D4000404601F00701B14207D90770006800F082
:100D50000700B04201D00120E7E72878400705D519
:100D60002068E96820F4E0500843206028780007F4
:100D700006D52068296920F4604040EAC10020605F
:100D800000F048F82168084AC1F30311515CC840DB
:100D90000649086006480068FFF7CEFE0020C4E759
:100DA000003C024008380240BE1600081400002033
:100DB0000C0000200F2202600C4A136803F00303AA
:100DC0004360136803F0F0038360136803F4E05397
:100DD000C36012684FF4E05303EAD2020261044890
:100DE000006800F007000860704700000838024003
:100DF000003C02400448054900680968044AC1F300
:100E00008221515CC840704714000020083802401D
:100E1000CE160008154810B5006810F00C021448F2
:100E200013D01449042A0FD0082A0ED10F4C241FC6
:100E30002268236802F03F025B0207D52068C0F3F6
:100E40008810A0FB010106E0084610BD2168C1F32F
:100E50008811A1FB00010023FFF706FA2168C1F306
:100E60000141491C4900B0FBF1F010BD08380240B7
:100E70000024F40040787D012DE9F84F04006ED085
:100E80002078DFF84C93C007A9F104054AD009F196
:100E900004000168C1F38101012908D00068C0F392
:100EA000810002280AD1D9F80000400206D528683E
:100EB000800337D560680028E1D033E06068B0F582
:100EC000803F10D0B0F5A02F286810D020F48030DB
:100ED0002860286820F4802028606068A8B1FFF7A7
:100EE00003FE06460DE0286840F48030F4E740F445
:100EF00080202860F7E700BFFFF7F6FD801B64281D
:100F000073D828688003F7D50CE0FFF7EDFD06469F
:100F100005E000BFFFF7E8FD801B6428F0D82868D3
:100F20008003F7D42078DFF8AC8280074FF0000A06
:100F30003ED5A748001D016811F00C0F08D00068CD
:100F4000C0F3810002280BD1D9F80000400207D479
:100F50002868800716D5E068012800D112E033E147
:100F6000E068B8B10120C8F80000FFF7BDFD0646F3
:100F700005E000BFFFF7B8FD801B0228C0D8286835
:100F80008007F7D52868216920F0F80040EAC10001
:100F900028600DE0C8F800A0FFF7A6FD064604E0B3
:100FA000FFF7A2FD801B02281FD828688007F7D40E
:100FB0002078000722D5864F87486169703771B164
:100FC00001210160FFF790FD064604E0FFF78CFD6C
:100FD000801B022809D838688007F7D50EE0C0F8D2
:100FE00000A0FFF781FD064605E082E0FFF77CFDEB
:100FF000801B02287DD838688007F7D42078400706
:1010000068D5DFF8CCB100270BF13C0BDBF8000012
:10101000C0000BD4DBF8001041F08051CBF8001079
:10102000DBF80000012700F0805000906B4E306824
:10103000C00510D4306840F480703060FFF754FD74
:10104000009005E0FFF750FD0099401A022850D8A3
:101050003068C005F6D55E4EA0686C3601280FD00A
:101060000528306810D020F001003060306820F092
:1010700004003060A068B8B1FFF736FD00900FE0C3
:10108000306840F00100F4E740F004003060F7E71A
:10109000FFF72AFD0099411A41F28830814266D853
:1010A00030688007F4D50EE0FFF71EFD009007E0E2
:1010B000FFF71AFD0099411A41F28830814256D853
:1010C00030688007F4D42FB1DBF8001021F0805194
:1010D000CBF80010A069C8B33D49091D0968C1F3E8
:1010E000810102294AD00228504607D0C8F8600082
:1010F00000E03CE0FFF7F8FC04463BE04746C8F858
:101100006000FFF7F1FC064605E000BFFFF7ECFCCE
:10111000801B02282BD828688001F7D4D4E9070166
:101120000843A16A2E4A490802EB0141626A41EA7A
:101130008211084394F82C1040EA0161C9F80010AC
:1011400001203866FFF7D0FC044606E03EE000BF11
:10115000FFF7CAFC001B022809D828688001F7D5D0
:1011600034E000BFFFF7C0FC001B022802D90320B7
:10117000BDE8F88F28688001F4D427E00128F7D073
:10118000D9F80000E26900F4800191421CD1226A82
:1011900000F03F01914217D147F6C071626A0140E9
:1011A000B1EB821F10D1A26A4FF0FF3300F440313F
:1011B00003EB5202B1EB024F06D194F82C1000F071
:1011C0007060B0EB016F01D00120D1E70020CFE7C4
:1011D0000438024000004742800E47420070004041
:1011E0000000FFFF7047704710B5040003D094F86B
:1011F0003D0010B107E0012010BD002084F83C0044
:10120000204600F01EF8022084F83D00211D2068D1
:1012100000F0D2F9012084F8460084F83E0084F8FA
:101220003F0084F8400084F8410084F8420084F8CC
:10123000430084F8440084F8450084F83D00002011
:1012400010BD704790F83D10012901D00120704772
:10125000022180F83D100168CA6842F00102CA60AC
:1012600000681149884214D0B0F1804F11D00F4965
:1012700088420ED00E4988420BD00E49884208D0D1
:101280000D49884205D00D49884202D00C49884258
:1012900004D1816801F00701062903D0016841F0FB
:1012A000010101600020704700000140000400407F
:1012B00000080040000C00400004014000400140D4
:1012C00000180040704770B50446006801694FF08F
:1012D0000005C943890715D4C168C943890711D4DA
:1012E000E91E01610120207720688069800720467F
:1012F00002D0FFF7E7FF04E000F098F8204600F086
:1013000096F8257720680169C943490717D4C16851
:10131000C943490713D46FF004010161022020770B
:101320002068806910F4407F204602D0FFF7CAFF92
:1013300004E000F07BF8204600F079F8257720687B
:101340000169C943090716D4C168C943090712D402
:101350006FF008010161042020772068C0698007D0
:10136000204602D0FFF7AEFF04E000F05FF8204611
:1013700000F05DF8257720680169C943C90617D4D4
:10138000C168C943C90613D46FF010010161082078
:1013900020772068C06910F4407F204602D0FFF714
:1013A00091FF04E000F042F8204600F040F8257775
:1013B00020680169C943C90708D1C168C943C90781
:1013C00004D1891E0161204600F032F820680169CD
:1013D000C943090609D4C168C943090605D46FF099
:1013E000800101612046FFF7FDFE20680169C943C5
:1013F000490609D4C168C943490605D46FF04001C4
:101400000161204600F01EF820680169C943890681
:101410000BD4C168C943890607D46FF0200101616C
:101420002046BDE87040FFF7DEBE70BD70477047D4
:1014300000680349884201D1FFF75CBB7047000098
:10144000000800407047FEE7174910B515480860CE
:1014500016480024802204704270E1228270C47019
:101460000471447148604FF400008860A1F1D80015
:10147000C860A038086140F2F45048610846FFF7A0
:1014800043F908B1FFF72CF9074838213838FEF73F
:1014900062FF05482121383801604FF44001C0E95E
:1014A000044110BD00800240900100200000002097
:1014B000114808B5016841F080010160016801F040
:1014C00080010091016841F004010160016801F0B0
:1014D00004010091016841F001010160016801F01F
:1014E00001010091016841F002010160006800F013
:1014F0000200009008BD000030380240FEE7FEE721
:10150000704770477047000030B593B0302168468F
:10151000FEF721FF14210CA8FEF71DFF1D48002532
:10152000016841F080510160006800F08050119026
:101530001948016841F4804101600068022400F408
:101540008040119001200390102004900094069494
:101550000820CDE90750A820CDE9090404200B900C
:101560006846FFF789FC08B172B6FEE70CA90F20A8
:1015700081E831004FF4A0500F904FF4805010904C
:1015800005210CA8FFF77CFB002801D072B6FEE70E
:1015900013B030BD4038024000700040024801687E
:1015A00041F470010160704788ED00E00148FFF7E9
:1015B0008ABE000040020020F0B50268254C264D8E
:1015C000264E274F274B4FF0804CA04209D0604554
:1015D00007D0A84205D0B04203D0B84201D098420B
:1015E00004D122F0700E4A6842EA0E02A0421BD0DB
:1015F000604519D0A84217D0B04215D0B84213D0D8
:10160000984211D0184DA8420ED0184DA8420BD0C8
:10161000174DA84208D0174DA84205D0164DA84234
:1016200002D0164DA84203D122F44075CA682A435D
:101630004D6922F080022A4302608A68C2620A6809
:101640008262A04201D0984201D10969016301215F
:101650004161F0BD0000014000040040000800406E
:10166000000C0040000401400040014000440140E3
:101670000048014000180040001C004000200040CD
:10168000FEE70907090E002804DB00F1E02080F8DE
:101690000014704700F00F0000F1E02080F8141DE6
:1016A0007047FFF72FFAFFF72FFFFFF701FFFFF754
:1016B000CBFEFEE74FF04070E1EE100A70470000ED
:1016C00000000000000001020304060708090000F2
:1016D0000000010203040000F816000800000020CA
:1016E00018000000C40100081017000818000020AE
:1016F000D0080000E0010008000000000000000029
:101700000100000010000000000000000024F400B0
:040000050800018965
:00000001FF
